:10000000C129A0007F39201B803C0920A01B003C97
:1000100008008A01820700340334063409340C34A2
:1000200010341334163419341C341F34223425345C
:1000300028342B342E3431343334363439343C3490
:100040003F3441344434473449344C344E345134D1
:100050005334553458345A345C345E34603462342A
:100060006434663468346A346B346D346F3470349D
:1000700071347334743475347634783479347A3432
:100080007A347B347C347D347D347E347E347E34EB
:100090007F347F347F347F34A0005E20A000732043
:1000A000A700A00A7320A600A00E7320A500A00A36
:1000B000732088202B08A3002A085E2900308A00BC
:1000C00020080F398207A6348034A034C03482342B
:1000D000A234C2348434A434C4348634C634E03404
:1000E000E234E434E63400308A0020080F39820715
:1000F0000234B93403340234033454340334AD3499
:100100000434B934053438340534C5340634613424
:10011000A4002508A402031CA5032708A602031CAB
:10012000A7033B09A2003909A300A20A0319A30AE5
:100130004130A900AC01AD01AE01AF01A8013A0800
:100140008400380939218413BD212408AC07031821
:10015000AD0A2508AD072608AE070318AF0A270821
:10016000AF072D080120803EA1002F080120803E0E
:10017000A107210CA80700083804031C38068000DA
:10018000290303194130A9000319A20A0319A30F77
:10019000A428BC29A6003A0884000930A70003104F
:1001A000D620A60CA70BD0280314D6288413B71D7D
:1001B000E52800083804371D380680008417000839
:1001C0003804031C38068000F02800083804031C9B
:1001D0003806371938068000841738098005F0285A
:1001E000370D0639A000F920A100A00AF92000006F
:1001F0006B2901308A0020080029FF3FFF3FFF3FA5
:1002000082070134993403343934003460340C34B7
:10021000FD34A3003A088400380939218413A30867
:100220000319BC29F030A50022088038A400F03062
:10023000A5030319A5000319A3030319BC2920086A
:10024000A6002108A70027306A212608A000270859
:10025000A1004921030120183808A21F3808A2086C
:1002600003190301A40F3629800614293729000039
:10027000172984178005BC2901308A00280807390E
:1002800082070134023404340834103420344034FA
:100290008034210820040319A00A8030201AA10606
:1002A0002019A106A018A106210DA00DA10DBC29A1
:1002B00083169B001C141A08BC29A301A200FF305E
:1002C000A207031CA307031CBC290330A100E630CE
:1002D0006B215F29A101FC3EA000A109031C762926
:1002E000FF300000A00703187129A0076400A10FC8
:1002F00070290800A8003C21A001A101A81DA000B0
:10030000A819A1002008BC29A0001130FF3EA00DB3
:10031000A10D031C8629BC290310A10CA00CFF3ED3
:1003200003188C292008BC29A2000530A800230846
:100330002102031D9D2922082002043003180130E8
:10034000031902302805031DFF30BC291030A80016
:10035000A101A001A70CA60C031CB4292208A00728
:1003600023080318230FA107A10CA00CA50CA40CB3
:10037000A80BAA292408BC29831303138312640041
:10038000080007309F008316073085008113831211
:10039000C1010508C1000330C1054108033C031C2D
:1003A000DC29D421BF00DC2901308A004108820702
:1003B0000734053404340634FA210530BA00043019
:1003C000B800C830BB00B9013230AA00AB013C080C
:1003D0004C200530BA001030B8007330A2000A304B
:1003E00009210530BA000830B8003F08B7003C08C2
:1003F000CA20C92932305D2186018316F03086007B
:1004000083120608A000A10104308F21B200210848
:10041000B3003208A0003308A100A3010F309421DB
:10042000031DFC2932305D21C0016400043040020C
:100430000318322A860140087A21B2002108B3004D
:10044000FF3032068316860083120608A000A10141
:1004500004308F21BD0064003D080F3C031D332A8A
:10046000C00F152A142A4008A600A7010430A200D4
:10047000A301A621B2002508B3000F303D06B40049
:100480000030B5003508A10034088421B400B5015E
:100490003208B40733080318013EB5073403BE0021
:1004A0003E085821BC0008006300542AFF3FFF3F6C
:1004B000FF3FFF3FFF3FFF3FFF3FFF3FFF3FFF3F4C
:1004C000FF3FFF3FFF3FFF3FFF3FFF3FFF3FFF3F3C
:1004D000FF3FFF3FFF3FFF3FFF3FFF3FFF3FFF3F2C
:1004E000FF3FFF3FFF3FFF3FFF3FFF3FFF3FFF3F1C
:02400E00623F0F
:104200000100020003000F000400050006000E007C
:104210000700080009000D000A0000000B000C0058
:10422000FF00FF00FF00FF00FF00FF00FF00FF0096
:10423000FF00FF00FF00FF00FF00FF00FF00FF0086
:10424000FF00FF00FF00FF00FF00FF00FF00FF0076
:10425000FF00FF00FF00FF00FF00FF00FF00FF0066
:10426000FF00FF00FF00FF00FF00FF00FF00FF0056
:10427000FF00FF00FF00FF00FF00FF00FF00FF0046
:10428000FF00FF00FF00FF00FF00FF00FF00FF0036
:10429000FF00FF00FF00FF00FF00FF00FF00FF0026
:1042A000FF00FF00FF00FF00FF00FF00FF00FF0016
:1042B000FF00FF00FF00FF00FF00FF00FF00FF0006
:1042C000FF00FF00FF00FF00FF00FF00FF00FF00F6
:1042D000FF00FF00FF00FF00FF00FF00FF00FF00E6
:1042E000FF00FF00FF00FF00FF00FF00FF00FF00D6
:1042F000FF00FF00FF00FF00FF00FF00FF00FF00C6
:00000001FF
